:1000000022C03BC03AC039C038C037C077C0C6C074
:1000100034C033C0E8C031C030C02FC02EC02DC0A6
:100020002CC02BC02AC030C126C128C118C131C183
:1000300019C11BC10BC12BC11BC123C10AC129C1DD
:100040000BC1280C010611241FBECFEDCDBF10E05F
:10005000A0E6B0E0ECEBF5E003C0C89531960D9258
:10006000A238B107D1F710E0A2E8B0E001C01D92BC
:10007000A839B107E1F77FD1A0C2C2CFBD9A969A45
:10008000C09AC29AC39A089582E08BB98CE089B96C
:1000900088E98AB908951DBC1CBC81E090E099BD37
:1000A00088BDBC9A8FB581628FBD8EB589608EBDCB
:1000B0000895459B0CC0A0E0B0E06BD2802D99273D
:1000C00088BD809194008F7E809394000895A1E074
:1000D000B0E05FD2802D992788BD80919400806127
:1000E00080939400089588E488B982E081B90895E6
:1000F00083E083BF89B7826089BF08951F920F9202
:100100000FB60F9211248F93869906C080919400A8
:1001100081608093940005C0809194008E7F8093CD
:100120009400B09906C080919400826080939400FE
:1001300005C0809194008D7F80939400B29906C091
:100140008091940084608093940005C08091940015
:100150008B7F80939400B39906C08091940088604F
:100160008093940005C080919400877F80939400D1
:100170008091940085FF02C0C59A01C0C598809106
:100180009500882329F080919500815080939500F7
:100190008F910F900FBE0F901F9018951F920F9286
:1001A0000FB60F9211248F939F93EF93FF9380913B
:1001B00096008F5F8093960080919600803110F0BA
:1001C00010929600809196009CB1E2E8F0E0E80F72
:1001D000F11D9083FF91EF919F918F910F900FBE32
:1001E0000F901F9018951F920F920FB60F92112427
:1001F0002F933F934F935F936F937F938F939F932F
:10020000AF93BF93EF93FF9354DFFF91EF91BF91B3
:10021000AF919F918F917F916F915F914F913F919E
:100220002F910F900FBE0F901F9018955D9BFECFE2
:100230008CB908959927AA27BB27F92FE82F319762
:10024000EE30F10530F5ED5EFF4F099480E3EEDF0F
:10025000089581E3EBDF089582E3E8DF089583E307
:10026000E5DF089584E3E2DF089585E3DFDF0895A5
:1002700086E3DCDF089587E3D9DF089588E3D6DFDE
:10028000089589E3D3DF08958AE0D0DF08958CE0F4
:10029000CDDF0895282F21502F3F41F0EAEFF0E005
:1002A0008E2F9F2F0197F1F72150D0F70895CF930C
:1002B000DF93D92FC82F8881882329F0219612D166
:1002C00088818823D9F7DF91CF91089561E081E09B
:1002D00016D180E690E0EBDF62E081E010D189E6A4
:1002E00090E0E5DF869BFECF8091940099278F7088
:1002F00090708930910529F18A30910534F4843069
:100300009105C1F00897A1F506C08C30910539F030
:100310000E9771F508C088B5815088BD29C088B591
:100320008F5F88BD25C0C598809194008F7D809394
:1003300094001EC0C59A80919400806280939400BE
:1003400017C080919400807FA3E0B0E0082E29D1EF
:100350008091940084FF06C088B5A1E0B0E0082E2B
:1003600020D1089588B5A0E0B0E0082E1AD10895F4
:1003700082E390DFB9CF1F9381DEC8D085DE8BDEAC
:10038000B2DEB6DEC59882E790E091DF62E081E000
:10039000B6D088E790E08BDF61E081E0B0D0A3E0E9
:1003A000B0E0F7D0802D807E809394007894869B77
:1003B0008DDF10929200109296001092930010E040
:1003C00001C010E080919600909193008917D1F1BF
:1003D000892F8F5F80939300803110F010929300EB
:1003E000E0919300FF27EE57FF4FE081E0939700E5
:1003F000EC3071F0ED3041F0EA3071F461E081E011
:100400007ED0109292001EC088E0809392001AC0A5
:100410006FD01092920016C080919200883019F42B
:1004200062E081E06CD0809197005CD08091920076
:100430008F5F80939200803128F01092920061E0EB
:1004400081E05DD08091940099278F709070892B06
:1004500009F4B7CF8091940099278F709070212F65
:1004600033278217930751F080919400182F1F7043
:10047000812FE0DE88E280939500A4CF80919500E3
:10048000882309F09FCF812FD5DE8AE080939500E5
:1004900099CF8A9A8B9A8C9A8D9AD09AD19A0895EC
:1004A0009298939894989598992780FD929A81FDB7
:1004B000939A82FD949A83FD959AD89A81E08A95C1
:1004C000F1F7D89808951F93182F82958F70E8DF61
:1004D000812FE6DF8DE08A95F1F71F910895D99A73
:1004E000F2DF0895FCDF0895D998EDDFD99A0895D9
:1004F00081E0FADF84EF91E00197F1F708958150F0
:10050000623009F4805C8068EFDF0895EF92FF921B
:100510000F931F93CF93DF93BCDF88E893E101979C
:10052000F1F7D898D99810E0C4EFD1E08C2F9D2F27
:100530000197F1F783E0B4DF1F5F1330B9F71DE0D7
:10054000812F8A95F1F782E0ABDF1A95F1F782E40B
:1005500090E0D92FC82F0F2EF4EFEF2EF1E0FF2EF1
:10056000F02D082F192F0D5F1F4FFD2FEC2FC89571
:10057000802DBADF9F2D8E2D0197F1F721960C1754
:100580001D0799F7DF91CF911F910F91FF90EF9089
:100590000895E199FECFBFBBAEBBE09A11960DB2B4
:1005A0000895E199FECFBFBBAEBB0DBA11960FB651
:0C05B000F894E29AE19A0FBE0895FFCF84
:1005BC00636F6E2E20302F3100206C656420322D3D
:1005CC00390073657475700063722B726573657492
:0205DC0000001D
:00000001FF
